:020000020000FC
:02000000FFC03F
:0200040076C2C2
:0200080075C2BF
:02000C007BC2B5
:020010007AC2B2
:0200140076C2B2
:0200180071C2B3
:02001C0070C2B0
:020020006FC2AD
:020024006AC2AE
:0200280077C29D
:02002C006DC2A3
:020030006CC2A0
:020034006BC29D
:0200380070C294
:02003C006BC295
:0200400068C294
:020044006BC28D
:0200480056C29E
:02004C0055C29B
:0200500066C286
:10020000F894FFE3EEEFC89501BE00E00BBB00E001
:100210000ABB00E008BB0FEF07BB03E005BB00EC27
:1002200004BB0FEF02BB0FEF01BBB0E0A0E600E0A4
:100230000D93B430E9F7A036D9F714E00FE51EBFEF
:100240000DBF00E005BF00E004BF00E000BF00E01C
:1002500003BF00E00CBF00E00FBD00E00EBD1FEFCC
:100260000FEF17BD06BD11E305E31BBD0ABD00E09E
:1002700005BD00E003BD00E207B907E006B910E0E4
:1002800003E010BD09B900E00BB900E00AB906E8C7
:1002900000BD00E00DB900E00EB902E400B900E0D5
:1002A00001B900EE0894001F02B900E006BF00E8A3
:1002B00008B90FE1102F01BD11BD00E00BBF00E038
:1002C00009BF0FEF08BF90E000E0009360000093CB
:1002D0006100009362000093630000936400009348
:1002E00065000093660000936700A895C09801E040
:1002F00026D100E015D1003430F4C098909A00E087
:100300000093600013C000916000013079F0C09A42
:10031000909801E014D100E003D10F3708F406C033
:10032000C098909A01E00093600000C0C19801E07D
:1003300006D101E0F5D0003430F4C198919A00E084
:100340000093610013C000916100013079F0C19AFF
:10035000919801E0F4D001E0E3D00F3708F406C033
:10036000C198919A01E00093610000C0C29801E039
:10037000E6D002E0D5D0003430F4C298929A00E082
:100380000093620013C000916200013079F0C29ABC
:10039000929801E0D4D002E0C3D00F3708F406C031
:1003A000C298929A01E00093620000C0C39801E0F5
:1003B000C6D003E0B5D0003430F4C398939A00E07F
:1003C0000093630013C000916300013079F0C39A79
:1003D000939801E0B4D003E0A3D00F3708F406C02F
:1003E000C398939A01E00093630000C0C49801E0B1
:1003F000A6D004E095D0003430F4C498949A00E07C
:100400000093640013C000916400013079F0C49A35
:10041000949801E094D004E083D00F3708F406C02C
:10042000C498949A01E00093640000C0C59801E06C
:1004300086D005E075D0003430F4C598959A00E078
:100440000093650013C000916500013079F0C59AF2
:10045000959801E074D005E063D00F3708F406C02A
:10046000C598959A01E00093650000C0C69801E028
:1004700066D006E055D0003430F4C698969A00E075
:100480000093660013C000916600013079F0C69AAF
:10049000969801E054D006E043D00F3708F406C028
:1004A000C698969A01E00093660000C0C79801E0E4
:1004B00046D007E035D0003430F4C798979A00E072
:1004C0000093670013C000916700013079F0C79A6C
:1004D000979801E034D007E023D00F3708F406C026
:1004E000C798979A01E00093670000C004E627D000
:1004F000FCCE189518951895189518951895189577
:100500001895189518951895189518951895189583
:100510001895189518951895189518951895189573
:100520001F9317B1107E102B17B916B1106C16B9A6
:1005300016B116FDFDCF04B105B11F9108951F93AB
:100540002F93A8952BE119E11A95F1F72A95D9F780
:0A0550000A95B9F72F911F91089545
:00000001FF
